:0E0000000207C52047534D323139200204B9A2
:0100130032BA
:01001B0032B2
:200023000205194154443E312A233B0D004154410D004154480D0041542B43504D533D22A1
:200043004D54222C224D45220D0041542B434D474C3D300D0041542B434D474C3D340D000D
:2000630041542B43434C4B3F0D0041542B435042523D310D0041542B435042523D320D008F
:2000830041542B434D47533D0041542B434D47573D0036310D00303031313030304238319A
:2000A3000030303034413832463443343934453344003044344635353534334400304435D3
:2000C3003235323344003230343334433344003044343134453344003230344235413344C8
:2000E3000032303230353133440041542B434D47533D0041542B434D47573D34350D003064
:20010300303131303030423831003030303441383146343735333444333233313339324564
:2001230034313533344432303244324430440038303030303030313030303030303030307C
:20014300303130323030303032313036323030303331383434303030313838433432303050
:20016300303843384332303038433438383430304337464638433030333746464638343157
:2001830031453030373138314443303033453030373830303143303033333831434330339B
:2001A300413434323235433643424135443336343442413544323234384241354431323412
:2001C300383434323231323438333831433132363830313830313633433032343033433087
:2001E3003430323430323030323032343034303031303234303830303043313833303030B6
:200203003033383143303030303037453030303030303030303030303030303030303030A0
:200223003030303030303038303030303030310038303030303030313030303030303030D9
:2002430030303030303030303030303030303030303034303343303030303633463830305A
:200263003036373745303630303733464337463030334646464646433031464646464645F4
:200283003046464646464630314646463033453033424645303343303033453030314330FA
:2002A300334230303030444336433738314533363434383432313232343933323443393269
:2002C300343842343244313234383738314531323638303138303136334330303030334362
:2002E30030343330304332303032304333303430303130334330383030304330303330308E
:2003030030303338314330303030303745303030303030303030303030303030303030309F
:200323003030303030303030383030303030303100383030303030303130453030303031C2
:2003430030333130303030313032323030303031303434303030303130343430303030337C
:2003630038343430303030454332323030303033383331314646383130304537464645319B
:20038300303030464646463030303146463746383030334645334643303033464331464300
:2003A300303342463030374443364330303030333634343030303032323438383234313197
:2003C300323438343432323132343833383143313236383031383031363343303030303398
:2003E30043303430383130323030323037453034303031303138303830303043303033308E
:2004030030303033383143303030303037453030303030303030303030303030303030309E
:200423003030303030303030303830303030303031003135310D003030353130303042380C
:200443003100303030344138383938333130383130300041545A0D004F4B004552524F5205
:20046300003E00312C22004B3A2200414E3D4D004B5A3D0054413D004C4E3D004F4E3D0097
:20048300433D0051313D0051323D0051343D0052494E4700324534330041453231005252FD
:2004A3003D00434C3D004F333D004F343D00534D3D00514F3D00C0E0C0D0C004758CB175DC
:2004C3008AE0E557600215571558E558200020A2E220010930021382E582E481ED20020863
:2004E30082E582E482E381EDA2E492B3B392825403701CE5B054F0FC655954F06011E5595E
:2005030054F0C44CC4120541E559540F4CF559D004D0D0D0E032C0E0C0D0309818C298E588
:2005230099B42002A13CB40D02A13CB40A02A13C120582A13CC299C203D0D0D0E032C00057
:20054300A85AF6055A7476B55A03755A6BD00022C000E55BB55A03E4A16CA85BE6F8055BD5
:200563007476B55B03755B6BE8D00022C000755A6B755B6BA85A760008B876FAD00022A9EE
:200583005CF7055CA95CB956167925E719F70909B957F8755C55155DA95DB92302055D22CB
:2005A300C000C2ACA85DE66002055DD2ACD00022C000C2AC755C24755D24A85C760008B898
:2005C30057FAD2ACD00022C0E0C4540F4430FD24C650032441FDD0E0540F443024C65003BC
:2005E300244122243A22E6B42201221205CACDC8CEC8F6E8CEF80EBE7F02E422CDC8CEC8E4
:20060300F6E8CEF80E08BE7FDDE422E6B4220122C8CEC8F6E8CEF80E08BE7FEFE422755708
:2006230064E55770FC222003FDF599D2032278247B00E66013EB936670090BEB93C3600B60
:2006430008C135087B00C135E824DB22783EC133E4936006120629A3C153227E11E6600E93
:200663001205CACD120629ED12062908DEEF741A120629227E047D0CE66039B42B0408E639
:20068300603208E6602EE61206291D74381206291D08E6601F08E6601B1206291D18E612B7
:2006A30006291D08DEEB74461206291D08E660041206291DED7001227446120629DDF922DF
:2006C300C0047433120629ECC413FC7430400274311206297433120629EC13FC7430400217
:2006E30074321206297433120629EC13FC7430400274331206297433120629EC13FC7430D8
:2007030040027434120629D00422B40007D200C2B3D28222B4FF07D200D2B3C28222B40111
:2007230007C200D201C20222B40207C200D202C20122B40F07C200D202D20122B4F0CEC273
:2007430000C202C20122E6B42C0D08E6540F75F00AA4082624D02208B87FEBC3227E24E6DB
:20076300B44F012230E6022409540FC4FC08E6B44F012230E6022409540F4CC8CEC8F6E8A4
:20078300CEF8080EE16278247B3E7C007F077D08E6C313CC13CCDF10CCC313C8CBC8F6C84A
:2007A300CBC8EC7C007F070BDDE77D0808EEB500DF22EBF87622783E7E241205E9EEF87686
:2007C3000022758107759870758921758DEF758BEF758780758CB1758AE0D28ED28CD2B925
:2007E30075A812740012070DC2031205B312056FE5B0440FF559C205C206C207C208D209E5
:20080300751F01D2AF74F012070D1206219004561206531205B312062190045B120631402C
:20082300A1709F90003A1206531205B312062190045B120631408B708990006D1206531257
:2008430005B3740012070D12062190046E120631400470E3D20690047B120631400408129A
:200863000D45900473120631400B08E6540F531FF0451FF51F9004A1120631400608B6419A
:2008830002D2059004A5120631400608B63102D20790047F120631400408120D2C75223030
:2008A3009004771206314003088622900483120631400408120D05900466120631403170FA
:2008C3002F087E5E12060E6025EEF876009000631206531205B374FF12070D12062190046D
:2008E3006A120631400A70087E6B0812060E01F60207C5740112070D9000F6120653120501
:20090300B312062190046412063140E470E2900102120653785E12067790010D120653784D
:200923006B12065E1205B312062112062190045B12063140BB70B91205B3E522B430022163
:200943007D740212070D75230A12062112062190049212063140127010E522B44312900086
:20096300351206531205B3217DE522B44302214CD523D61522E522B430C775236412056FC6
:20098300740112070D120553FC604B300703120CE374FF12070D30052A30081DE5596C5422
:2009A3000F6004D2E721B2E559FCC46C540FFC120D865017120D8621CE120BF9500D120B3C
:2009C300F921CE120E3E5003120E3E1205B312062112062121D91205B312062190049212AC
:2009E300063140197017740212070D9000353006039000301206531205B312062190004D38
:200A03002090039000581206531205B312062190045B120631404D704B90049C1206314091
:200A2300127041181818120760120789EBF87600020A559004971206314029702718181817
:200A4300120760EEF8762278277E3E12060EEEF876009004B112064F4012700808B6500734
:200A6300D208416F020B43B65402C2089004A112064F400F70EE08B64104D2054186B650D3
:200A8300EBC2059004A512064F400F70D708B63004C207419DB63102D2079004B512064F60
:200AA300400F70C008B63004C20941B4B63102D2099004AD12064F400F70A908B63004C27A
:200AC3008741CBB63102D2879004A912064F400F709208B63004C28641E2B631EBD2869032
:200AE300047312064F4037705708B63005531FF06121B63108531FF0431F016121B63208DA
:200B0300531FF0431F026121B63408531FF0431F046121B63808531FF0431F086121740F87
:200B230012070DE58044F0C4FCE5B044F05CFC120BF95003120BF91205B312062112062157
:200B4300D523267523649000631206531205B3740012070D12062190046A120631400A707C
:200B6300081207495003B522160209830207C5E52255036076616CE5225501606E616CF57D
:200B83002230094F9000781206531205B374FF12070D120621900486120631400D7034083D
:200BA300E52228F8E6120D3C61D690048A120631400D08E522C31328F8E6120D3C61D690D2
:200BC300048E120631400C08E522C3131328F8E6120D3CE51F540F609013400F13409813DB
:200BE300408D13500EE52255077008740212070D120CE302098390008C20B2039000831298
:200C030006531205B390009512065312062190046412063140657063900099120653785EC2
:200C23001206779000A41206531206C374331206297445120629ECC4FC1206C3AC80900083
:200C4300B51206531206C39000E412065330090C74351206297439120629816974341206F0
:200C63002974451206299000C012065330050E74341206297431120629818AD322743512C6
:200C8300062974301206299000C912065330070C7433120629743112062981A9743312067F
:200CA3002974301206299000D212065330060C7435120629743212062981C8743412062911
:200CC30074441206299000DB1206537433120629E51F540F4430120629741A120629C3228A
:200CE3009000261206531205B31206211206211206211206219000351206531205B3120610
:200D03002122B64102D20508B63102D20708B64D02D20608E6540F531FF0451FF51F0812C9
:200D23000D45C20808120D2C22120D541392841392851392861392872230E6022409540F38
:200D4300A12F120D5444F043590F5559F559D208227400B63003C3A160B63126D33308B684
:200D63003003C3A16CB6311AD33308B63003C3A178B6310ED33308B63003C3A184B63102DC
:200D8300D3332290008C20B2039000831206531205B3900435120653120621900464120672
:200DA30031403D703B90043A120653785E120677900445120653EC90013220E70990023371
:200DC30020050390033412065374301206297444120629ECC4FC1206C3741A120629C3229D
:200DE300D32208E6C408D622F87433120629E8C4540F44301206297433120629E8540F442E
:200E0300301206292241542B434D47573D35300D00303031313030304238310030303034DE
:200E230041383234003230343934453344003230344635353534334400D3229000631206EB
:200E4300531205B374FF12070D12062190046A12063140E570E3120DE5F57F08120DE5F568
:200E63007E08120DE5F57D08120DE5F57B08120DE5F57C740012070D900E081206531205B8
:200E8300B312062190046412063140AD70AB900E14120653785E120677900E1F120653E58B
:200EA3007B120DEB74331206297441120629E57C120DEB74321206297430120629E57D1221
:200EC3000DEB74321206297445120629E57E120DEB74321206297445120629E57F120DEB7A
:200EE300900E281206531206C374331206297445120629ECC4FC1206C3AC80900E31120667
:0B0F0300531206C3741A120629C32201
:00000001FF
